:0300000002313C8E
:0C313C0078FFE4F6D8FD7581690231834C
:100EC50020000A3C2E2E2E3E004950436F6E6E6563
:100ED50063745245510A004950436F6E6E656374E1
:100EE500000A49504E6F41434B210A003E432C56A0
:100EF5002C43432CC0E4E0EFF2E5F020D1E8EDEA25
:100F0500EEEC49500A003E432C4D41432C2530322E
:100F150062583A25303262583A25303262583A25BD
:100F2500303262583A25303262583A2530326258AA
:100F35002C4D414320E0E4F0E5F10A003E432C56F8
:100F450045522C20332E3220EEF2202573202573B6
:100F55002CC2E5F0F1E8FF20495020ECEEE4F3EB7C
:100F6500FF0A0041707220313820323030380031AC
:100F7500303A35383A3332003E432C4C442C5052EB
:100F85004F473A20202020202020202020202020EC
:100F9500202020202020202020202020202020204C
:100FA500202020202020202020202020202020203C
:100FB500202020202020202020202020202020202C
:100FC50020202020202020202CC4E0F2E020EFF07B
:100FD500EEF8E8E2EAE828F4E0E9EB290A003E2A1F
:100FE5002C312CCEF1EDEEE2EDFBE520EFE0F0E06B
:100FF500ECE5F2F0FB20F1E5F2E5E2EEE3EE20E8C8
:10100500EDF2E5F0F4E5E9F1E00A003E412C41306E
:10101500312C2562752E2562752E2562752E256269
:10102500752C495020E0E4F0E5F120E0E4E0EFF232
:10103500E5F0E00A003E412C4130322C2562752E48
:101045002562752E2562752E2562752C495020E086
:10105500E4F0E5F120EEF1ED2E20F1E5F0E2E5F02A
:10106500E00A003E412C4130332C2562752E256265
:10107500752E2562752E2562752C495020E0E4F009
:10108500E5F120F0E5E72E20F1E5F0E2E5F0E00AF4
:10109500003E412C4130342C2562752E2562752E7B
:1010A5002562752E2562752CCCE0F1EAE020F1E58C
:1010B500F2E80A003E412C4130352C2562752E257B
:1010C50062752E2562752E2562752CD8EBFEE70A12
:1010D500003E2A2C312CC4EEEF2E20EFE0F0E0ECA0
:1010E500E5F2F0FB20F1E5F2E5E2EEE3EE20E8EDD6
:1010F500F2E5F0F4E5E9F1E00A003E422C53303127
:101105002C2562752CC6E4E0F2FC20E7E0EFF0EE5A
:10111500F1E020F1EEE5E4E8EDE5EDE8FF20EEF2A3
:1011250020F1E5F0E2E5F0E00A003E422C533032D2
:101135002C2562752CCEE1ECE5ED20F120F1E5F0F2
:10114500E2E5F0EEEC20E1E5E720EAE2E8F2E0EDA9
:10115500F6E8E90A003E422C5330332C2562752C03
:10116500CFE5F0E5E7E0EFF3F1EA20EFF0E820EF77
:10117500EEF2E5F0E520F1E2FFE7E820F120F1E508
:10118500F0E2E5F0EEEC0A003E454E440A000A4462
:10119500756D7058202020202030302030312030CF
:1011A500322030332030342030352030362030376F
:1011B5002030382030392030412030422030432043
:1011C5003044203045203046000A3A003A20000AD3
:1011D500000A44756D7044202020202030302030D6
:1011E5003120303220303320303420303520303635
:1011F500203037203038203039203041203042200F
:10120500304320304420304520304600457272205E
:101215006B657900526420656570726F6D0A0052C6
:1012250064204D454D0A00526420436F64650A00F1
:10123500577269746520436F64650A004465627579
:10124500674950204F4E0A00446562756749502032
:101255004F46460A00446562756755736572204FAF
:101265006E0A00446562756755736572204F464680
:101275000A0044656275674D7367204F6E0A004426
:10128500656275674D7367204F46460A00436F6E6A
:10129500666967206C6F636B210A0057722065656C
:1012A50070726F6D0A0020536176652065657072F6
:1012B5006F6D210A00457272204D414321004C6F2C
:1012C50061643E3E002A003C4130313D003C4130E6
:1012D500323D003C4130333D003C4130343D003C23
:1012E5004130353D003C21003C5330313D003C53FD
:1012F50030323D003C5330333D003C5330353D00EA
:061305003C5330363D00B0
:063BC600010B00010900E3
:103BB600C28E438910758BFF758DB7D2ABD28E221C
:03001B000230AC04
:1030AC00C0E0C083C082C0D0C28E758BFF758DB757
:1030BC0020060675A61E75A6E10509D202E50B6071
:1030CC0002050BE50AD394014002150A050EE50E24
:1030DC00540F7048D20EE50E543F7012D200906619
:1030EC008BE0600A04F0E0D394B44002D206906600
:1030FC0086E0600204F0906104E0600214F09066D7
:10310C008CE0D394014003E014F0300502050CE58B
:10311C000DD394644004D2068002050DE508D394C7
:10312C000140021508D28ED0D0D082D083D0E032AC
:10086300C2AFC291C290D2B5C20B7D027C007F079A
:10087300123B6C8F49E549646060097D017F60121A
:100883003A9ED20BE4FDFC7F0B123B6C8F49E5498A
:1008930030E6097D04E4FF123AC2D20B7D017C00ED
:1008A3007F07123B6C8F49E5497008FD7FFF123AC1
:1008B3009ED20B300B03126000C288C2A8C2AA7575
:1008C30089001234E890633EE0B4FA06A3E064CEF4
:1008D300607BE4F54974362549F582E43463F58396
:1008E300E4F00549E549B443EC90633E74FAF0A3A0
:1008F30074CEF0A374CCF0906344740AF0E4A3F0D4
:10090300A304F0A3F090633A74FFF0A3F0A3F0E420
:10091300A3F0906355740AF0E4F549E5492401FF17
:10092300E433FE74362549F582E43463F583E0FD50
:10093300123A7A0549E549C3944340DFE4F5A775C4
:10094300A61E75A6E1907FF0F0A3F080FE906349A8
:100953007403F0A374CCF0E4906348F0122D38C212
:10096300B51236C4C206123915D20BC20DC20C9091
:1009730065767408F09062B47424F0E4A3F0906395
:100983003EE09062B6F090633FE09062B7F0906310
:1009930040E09062B8F0906341E09062B9F09063F8
:1009A30042E09062BAF0906343E09062BBF0750A54
:1009B30001E4906577F0C207C208C209C20A123A7D
:1009C300E6200B19AF497E007D03122AACE4FF1227
:1009D3002EC57E0E7FC5E4FBFDFC1227B990668B06
:1009E300E060037401F0E4906104F0F50C90657528
:1009F300F0F50D123BB675A70775A61E75A6E1D2D5
:100A0300AFE4F50D906104E0700312166790668CF5
:100A1300E0B401119080007410F0E490668CF0D281
:100A23000BC20CC20D908008E0F54930E405D207F3
:100A33007410F0E54930E508D2099080087420F07D
:100A4300E54930E608D2089080087440F0E50CC30D
:100A530094034019908002E4F0908001F0908000AC
:100A6300F0E50C94064006E4F50C1239159080A0CD
:100A7300E070031235669080B8E070031235E090A1
:100A830080D0E07003123792908000E0701330073B
:100A9300101228C0906331EFF0D39400400312008A
:100AA30036908002E07006908000E06005D2050277
:100AB3000A04C205E4F50C906104E06003020A0431
:100AC300200B12906578E0600C7E0E7FC71229C45C
:100AD300E4906578F03009121223E7906331EFF068
:100AE300D394004005E0FF12002F200803020C6D91
:100AF3001220DF906331EFF07003020A04906375F4
:100B0300E054BF247F7003020BD6147003020BAEB4
:100B130024026003020C0F200B077E0E7FCE1229E6
:100B2300C4200F03020C6D90634DE0700690635177
:100B3300E06067906682E0FF90634DE0B507249024
:100B43006683E0FE90634EE0B50618906684E0FE8F
:100B530090634FE0B5060C906685E0FE906350E02D
:100B63006E6037906351E06F6003020C6D90668393
:100B7300E0FF906352E06F6003020C6D906684E0C7
:100B8300FF906353E06F6003020C6D906685E0FF96
:100B9300906354E06F6003020C6DC2039065777439
:100BA30001F0120022750A01020C6D90668BE06061
:100BB300037401F090667AE0FF906377E06F60035F
:100BC300020C6D90667AE004F0E4F50A906575F026
:100BD300020C6D300303020C6D906344E07003025A
:100BE3000A04906355740AF0123BCDD203E4F50A6C
:100BF300906575F090668604F0E4906679F0A3F052
:100C0300200B677E0E7FDC1229C4805E90668BE02A
:100C130060037401F0300352906375E020E74B905A
:100C23006377E0FF906679E0FE6F600D906681E088
:100C33007007EE146F70338013906679E004F090C0
:100C43006331E0FFD3940440031226939060007451
:100C530082F0A37401F0906377E0906002F07E600D
:100C63007F007D0312324F020A04200303020D8525
:100C7300E50A706812365AEF60237E647F759064CC
:100C830076E02404FD12324F906681E07009906390
:100C930055E0F50A020A04E4F50A020A049066869E
:100CA300E0D3943C4036906681E0703090668604D1
:100CB300F0120032E4906475F0A37412F090667A37
:100CC300E0906477F0A374FDF090610563A2019056
:100CD300647963A2017F12121C70809E123BA38F62
:100CE30049E549B401159060007483F0E4A3F07EF4
:100CF300607F007D0212324F020A04E549D394015A
:100D0300401C9060007483F0A37401F0E54924FE55
:100D1300A3F07E607F007D0312324F020A04E50ACE
:100D230064016003020A04906575E004F0200B0778
:100D33007E0E7FE61229C4906355E0C394C8500425
:100D4300E02432F0906575E0C39405400DC203E4DE
:100D5300906577F0120022020A047C667D8290631C
:100D630049E0FAA3E0FB7F021233E07E647F7590D3
:100D73006476E02404FD12324F906355E0F50A02D5
:100D83000A04E50A64016003020A04906577E0142B
:100D9300604624FE6042147003020E78240460034C
:100DA300020A04E4F50C200F139065777404F090A5
:100DB3006575E05401F0750A01020A04908002741B
:100DC30010F0E4906577F090657504F0750AFA9079
:100DD300668274FFF0020A04906682E07003020EDA
:100DE300629064757480F09064777401F0E4A3F00A
:100DF300A304F0A37430F0A3747BF0E4F549747C8E
:100E03002549F582E43464F583747DF0747D2549C6
:100E1300F582E43464F583E4F0E5492407906476CD
:100E2300F07C667D82906349E0FAA3E0FB7F0212C7
:100E330033E07E647F75E5492409FD12324F9066E5
:100E430081E0601B123BCDD203E4F50A906575F097
:100E530090668604F0E4906679F0A3F0020A043009
:100E63000F07E4906577F080069065777404F0755A
:100E73000AFA020A049080027410F0750A0590655C
:100E830075E06401FFF09065777401F0EF701990DD
:100E93006351E06013FCA3E0FDA3E0FEA3E0FF9039
:100EA3006682121A11020A0490634DE0FCA3E0FD6E
:100EB300A3E0FEA3E0FF906682121A11020A0480E7
:010EC300FE30
:010EC400220B
:10003600906376E0B444047F0180027F009063758C
:10004600E0B447047E0180027E00EE5F604A906362
:100056003EE0906377F090633FE0906378F09063C2
:1000660040E0906379F0906341E090637AF09063AA
:1000760042E090637BF0906343E090637CF0906392
:10008600767452F09062AE63A2019080A863A201DA
:100096007F06121C70020859906331E0C394085021
:1000A6000302086290633EE0FF906377E06F6003AF
:1000B60002086290633FE0FF906378E06F6003029E
:1000C6000862906340E0FF906379E06F6003020886
:1000D60062906341E0FF90637AE06F60030208621A
:1000E600906342E0FF90637BE06F600302086290DA
:1000F6006343E0FF90637CE06F60030208629063F5
:1001060076E0B444159062AEE0B4FF0E63A20190AF
:1001160080A863A2017F06121C7090668BE06003C4
:100126007401F090668C7464F09063767452F0906B
:100136006375E0646D60030202637BFF7A0E79F1FA
:1001460012136D7BFF7A0F790B90633EE0F552A395
:10015600E0F553A3E0F554A3E0F555A3E0F556A367
:10016600E0F55712136D7552FF75530F7554687588
:1001760055FF75560F7557747BFF7A0F7941121329
:100186006D7BFF7A0F797D12136D7BFF7A0F79E312
:1001960012136D7BFF7A107910906344E0F552A339
:1001A600E0F553A3E0F554A3E0F55512136D7BFF7C
:1001B6007A10793A90634DE0F552A3E0F553A3E047
:1001C600F554A3E0F55512136D7BFF7A107968900C
:1001D6006351E0F552A3E0F553A3E0F554A3E0F52F
:1001E6005512136D7BFF7A10799690633AE0F552BB
:1001F600A3E0F553A3E0F554A3E0F55512136D7B88
:10020600FF7A1079B9906336E0F552A3E0F553A36F
:10021600E0F554A3E0F55512136D7BFF7A1079D6FD
:1002260012136D7BFF7A1079FFA20FE433F5521299
:10023600136D7BFF7A11792F906681E0F5521213C8
:100246006D7BFF7A11795A90668BE0F55212136D29
:10025600122F757BFF7A11798D12136D22906375BB
:10026600E0644C70737E117F93FBFDFC1227B990FE
:10027600637DE0F54AA3E0F54BE4F54DE54A90636E
:100286007FF0A3E54BF07E117FCE7C637D7F7B0202
:100296001227B9E4F54C854B82854A83E0FF747FCB
:1002A600254CF582E43463F583EFF0054BE54B709E
:1002B60002054A054CE54CB410DC7E117FD17C6307
:1002C6007D7F7B101227B9054DE54DC3941040ACD8
:1002D6007E117FD41229C422906375E0646C70602D
:1002E600F54E7E117FD6FBFDFC1227B9E4F54DE4F1
:1002F60090637FF0A3E54EF07E117FCE7C637D7F19
:100306007B021227B9E4F54CA84EE6FF747F254C14
:10031600F582E43463F583EFF0054E054CE54CB405
:1003260010E67E117FD17C637D7F7B101227B90595
:100336004DE54DC3940840B77E117FD41229C422DF
:10034600906375E0644B7061F54C7467254CF582DB
:10035600E43463F583E060327467254CF582E43457
:1003660063F583E0F460237467254CF582E4346317
:10037600F583E0FF747D254CF582E43463F583E074
:10038600B50710054CE54CB408C09061047432F012
:100396000208599063757421F0300B030208597EE8
:1003A600127F111229C4020859906375E0B4521ADB
:1003B600200B077E127F191229C49063757472F0A0
:1003C6007E637F757D081231C822906375E06449AB
:1003D6007045200B077E127F241229C490637DE0AE
:1003E600F54AA3E0F54BE4F54C854B82854A83E05C
:1003F600FF747F254CF582E43463F583EFF0054BFB
:10040600E54B7002054A054CE54CB480DC7E637F03
:10041600757D8A1231C822906375E0644370462068
:100426000B077E127F2C1229C490637DE0F54AA348
:10043600E0F54BE4F54C854B82854A83E493FF74E3
:100446007F254CF582E43463F583EFF0054BE54BED
:100456007002054A054CE54CB480DB7E637F757DF2
:100466008A1231C822906375E0645A7053200B07D4
:100476007E127F351229C490637DE0F54AA3E0F52C
:100486004B7C637D7F7B80AF4BAE4A1239EDE4F542
:100496004C854B82854A83E493FF747F254CF58215
:1004A600E43463F583EFF0054BE54B7002054A052E
:1004B6004CE54CB480DB7E637F757D8A1231C822A1
:1004C600906375E06444600302055790637DE0FF26
:1004D60064447003020859EFB4310CC20B7E127FDC
:1004E600411229C402085990637DE0B4300CD20B46
:1004F6007E127F4D1229C402085990637DE0B43202
:100506000CD20C7E127F5A1229C402085990637DC0
:10051600E0B4330CC20C7E127F681229C40208595B
:1005260090637DE0B4340CD20D7E127F771229C41D
:1005360002085990637DE0B4350CC20D7E127F84AB
:100546001229C402085990637DE0FF12001E0208BA
:1005560059906104E07013200B077E127F921229D6
:10056600C49063757421F00208599061047432F0E6
:10057600906375E0FFB45104C2AF80FEEF6457701C
:1005860045200B077E127FA01229C490637EE0905F
:100596006331F0E4F54C906331E0FFE54CC39F40D6
:1005A60003020859747F254CF582E43463F583E031
:1005B600FF90637DE0254C24ADF582E43461F5833C
:1005C600EFF0054C80D0906375E06453600302063B
:1005D6007A200B077E127FAB1229C490633EE0FFA0
:1005E6009061B6E06F703C90633FE0FF9061B7E0CA
:1005F6006F7030906340E0FF9061B8E0B5072490DB
:100606006341E0FF9061B9E0B50718906342E0FFEF
:100616009061BAE0B5070C906343E0FF9061BBE0E0
:100626006F60169063757421F0300B030208597ED3
:10063600127FBA1229C4020859E4F54CE4F50DAF4D
:100646004CFE74AD254CF582E43461F583E0FD1271
:100656003A7A054CE54CC394FE40E1C2AFE4907F84
:10066600F0F0A3F0907FFD74AAF0A374FFF0A374DA
:1006760055F080FE906375E0644F704C90637DE0AA
:10068600F54AA3E0F54BE54B454A700A200B077E79
:10069600127FC31229C4200B077E127FCA1229C4F7
:1006A600E4F54C747F254CF582E43463F583E085EC
:1006B6004B82854A83F0054BE54B7002054A054C93
:1006C600E54CB480DE020859906375E0FFB445211D
:1006D60090637DE0FDA3E0907FF0CDF0A3EDF0C246
:1006E600AF907FFD74AAF0A374FFF0A37455F08059
:1006F600FEEF6465600302086290637DE0FFA3E09D
:10070600907FF0CFF0A3EFF0E4F54AF54BD3907F5E
:10071600F1E0954B907FF0E0954A4020E4F50D25F9
:100726004BFFE54A3401FE854B82854A83E0FD1284
:100736003A7A054BE54B7002054A80D17E127FCC92
:100746001232D6EF4E6020120003906344EFF0128F
:100756000003906345EFF0120003906346EFF0123A
:100766000003906347EFF07E127FD21232D6EF4E2F
:10077600602012000390634DEFF012000390634E69
:10078600EFF012000390634FEFF0120003906350F6
:10079600EFF07E127FD81232D6EF4E6020120003A1
:1007A600906351EFF0120003906352EFF0120003D2
:1007B600906353EFF0120003906354EFF07E127FC4
:1007C600DE1232D6EF4E602012000390633AEFF04D
:1007D60012000390633BEFF012000390633CEFF0CE
:1007E60012000390633DEFF07E127FE41232D6EFE3
:1007F6004E6020120003906336EFF0120003906300
:1008060037EFF0120003906338EFF01200039063A5
:1008160039EFF0E4F54CE4F50DE54C2401FFE43343
:10082600FE7436254CF582E43463F583E0FD123A16
:100836007A054CE54CC3944340DCC2AFE4907FF0AC
:10084600F0A3F0907FFD74AAF0A374FFF0A3745593
:0C085600F080FE7E637F757D081231C8C3
:010862002273
:1039B500AE07EEC39430400BEED394395005EE2498
:1039C500D0FF22EEC39461400BEED394665005EE12
:1039D50024A9FF22EEC39441400BEED39446500533
:0839E500EE24C9FF22AF062207
:103B89009062ADE004F070069062ACE004F09062DF
:0A3B9900ACE0FEA3E0FF123B4F2258
:10000300123B891239B5EFC454F0FEC006123B8986
:080013001239B5D0E02FFF22E5
:1038B800E4906A0EF0123B89906A0FEFF0C39430DF
:1038C8004018E0FFD394395011906A0EE02405F5B2
:1038D80082E43461F583EFF08011906A0EE02405EC
:1038E800F582E43461F583E4F0800C906A0EE0041C
:1038F800F0E0D3940840BE754D00754E00754F003A
:0C390800E4F5507B017A617905121F3B49
:013914002290
:0432D6008E4F8F5038
:1032DA009062ACE4F0A374FFF0123B89EF606EF4E5
:1032EA00606B855082854F83E493B507EC75510175
:1032FA00E5502551F582E4354FF583E49360259036
:10330A0062ADE02551FF9062ACE03400FE123B4F03
:10331A00E5502551F582E4354FF583E493B507046A
:10332A00055180CCE5502551F582E4354FF583E40B
:10333A009370A6E55124FFFFE434FFFE9062ADE0EE
:10334A002FF09062ACE03EF07E007F0122E4FEFFA7
:01335A002250
:102D38007E127FEA1232D6EF4E70037F01227E1296
:102D48007FED1232D6EF4E600C123B89EF24D0246F
:102D5800FF920F8002D20F7E127FF31232D6EF4E0F
:102D6800600C123B89EF24D0906681F08005E490D6
:102D78006681F07E127FF91232D6EF4E600C123B5C
:102D880089EF24D090668BF08005E490668BF07E06
:102D9800127FFF1232D6EF4E600C123B89EF24D01F
:102DA80024FF92018002C20190633E63A2019066F3
:102DB8007B63A2017F06121C7030013B7E137F05E6
:102DC8001232D6EF4E603012000390667BEFF0129D
:102DD800000390667CEFF012000390667DEFF0121E
:102DE800000390667EEFF012000390667FEFF0120A
:0A2DF8000003906680EFF07F0022D8
:10396E00906576E0C3947C503D906576E0FE04F061
:10397E0074B42EF582E43462F583EFF0BF0A27901B
:10398E006576E0FF04F074B42FF582E43462F583BB
:10399E00E4F0906576E0FF12335B9065767408F084
:0739AE009062B5E004F02275
:103915009080007480F090633663A201F583F58290
:1039250063A2017F08121C7090633E63A201908020
:103935008863A2017F0A121C70908092E4F0A37440
:1039450032F0A37401F0906348E0FF9080B1F090ED
:1039550080E1EFF09080957455F0A3F090800074AD
:0939650001F090800974F0F022D9
:10356600908009E04410F09080A0E0706C9080A1FB
:103576007482F09080A874FFF0A3F0A3F0A3F07F0C
:10358600039080AEEFF07FCBA3EFF07F039080AC8B
:10359600EFF0A374CBF09080007402F0906A0212F0
:1035A6001A1D00000000906A02E0908040F0906AC8
:1035B60003E0908041F0906A04E0908042F0906AC7
:1035C60005E0908043F0A3E4F0A3F0A3F0A3F0900D
:0935D6008018F0A3F0A3F0A3F0AB
:0135DF0022C9
:10379200908009E04440F09080D17482F0906349B7
:1037A200E0FF9080DEF090634AE0FF9080DFF090CF
:1037B20080027402F0906A06121A1D000000009046
:1037C2006A06E0908058F0906A07E0908059F09085
:1037D2006A08E090805AF0906A09E090805BF0A35A
:1037E200E4F0A3F0A3F0A3F0908030F0A3F0A3F0F4
:0237F200A3F042
:0137F40022B2
:1035E000908009E04420F09080B8E0706C9080B941
:1035F0007482F07F039080C6EFF07FCDA3EFF07F61
:10360000039080C4EFF0A374CDF09080C074FFF0FD
:10361000A3F0A3F0A3F09080017402F0906A0A1264
:103620001A1D00000000906A0AE090804CF0906A39
:103630000BE090804DF0906A0CE090804EF0906A24
:103640000DE090804FF0A3E4F0A3F0A3F0A3F0907E
:093650008024F0A3F0A3F0A3F024
:01365900224E
:1033E0008C4A8D4BA907EAFDE975F018A424ACFFBF
:1033F000E5F034808F82F583EDF0EBFDE975F01890
:10340000A4FFAEF024ACFBEE34808B82F583A3EDF9
:10341000F0854B828C83E0FDEF24A8FFEE3480FE24
:103420008F82F583EDF0854B828C83A3E08F828EB3
:1034300083A3F0854B82854A83A3A3E0FDE975F061
:1034400018A424A8FFE5F03480FE8F82F583A3A39F
:10345000EDF0854B828C83A3A3A3E08F828E83A3A0
:04346000A3A3F02210
:0631C8008D4FAB07AA06C3
:1031CE00908000E030E5079065787401F022906AF7
:1031DE0002E0FCA3E0FDA3E0FEA3E0F5538E528DCA
:1031EE00518C50AE02AF038E838F8263A201E552E3
:1031FE00540744C0F58385538263A201AF4F121C5E
:10320E00E2E4FCFDFEE553254FF553EE3552F55243
:10321E00ED3551F551EC3550F550908040E550F0BC
:10322E00A3E551F0A3E552F0A3E553F090800074AE
:10323E0020F0AF53AE52AD51AC50906A02121A113B
:01324E00225D
:06324F008D4AAB07AA0640
:10325500908002E030E5079065787403F022906A6B
:1032650006E0FCA3E0FDA3E0FEA3E0F54E8E4D8D48
:103275004C8C4BAE02AF038E838F8263A201E54D6A
:10328500540744D0F583854E8263A201AF4A121CD0
:10329500E2E4FCFDFEE54E254AF54EEE354DF54DD5
:1032A500ED354CF54CEC354BF54B908058E54BF036
:1032B500A3E54CF0A3E54DF0A3E54EF09080027434
:1032C50020F0AF4EAE4DAD4CAC4B906A06121A11C4
:0132D50022D6
:022EC5008F4A32
:102EC700908001E030E5099065787402F07F002278
:102ED700906A0AE0FCA3E0FDA3E0FEA3E0F54E8EB6
:102EE7004D8D4C8C4B90667B63A201E54D54074496
:102EF700C8F583854E8263A2017F06121CF8E54E52
:102F07002406F54EE4354DF54DE4354CF54CE435E6
:102F17004BF54B90657963A201E54D540744C8F51D
:102F270083854E8263A201AF4A121CF8E4FCFDFEC2
:102F3700E54E254AF54EEE354DF54DED354CF54C44
:102F4700EC354BF54B90804CE54BF0A3E54CF0A3EB
:102F5700E54DF0A3E54EF09080017420F0AF4EAE42
:0D2F67004DAD4CAC4B906A0A121A11AF4AE6
:012F7400223A
:1028C0009081E0E0F54A054A054A054A054A054A6D
:1028D000054A054A054A054A054A908010E0F54D2B
:1028E000A3E0F54EA3E0F54FA3E0F5509081E1E0C1
:1028F000F54A054A054A054A054A054A054A054A70
:10290000054A054A054A908014E0F551A3E0F552C6
:10291000A3E0F553A3E0F554E553B54F08E554B5EE
:1029200050037F0022E4F54AE553540744E0F58361
:1029300085548263A20190637563A2017F08121D12
:102940002890637763A2019062AE63A2017F0612B2
:102950001C70906375E0F54BA3E0F54CE4F54A90EC
:102960006375E0702AA3E024F8F54AE55354074460
:10297000E0F58385548274082582F582E43583F579
:102980008363A20190637563A201AF4A121D28AE52
:102990004BE4FCFDE554254CF554E5533EF553ED71
:1029A0003552F552EC3551F551908014E551F0A3B4
:1029B000E552F0A3E553F0A3E554F0908000744095
:0329C000F0AF4A2B
:0129C30022F1
:1020DF009081E6E0F54A054A054A054A054A054A50
:1020EF00054A054A054A054A054A908028E0F54DFC
:1020FF00A3E0F54EA3E0F54FA3E0F5509081E7E0A4
:10210F00F54A054A054A054A054A054A054A054A58
:10211F00054A054A054A90802CE0F551A3E0F55297
:10212F00A3E0F553A3E0F554E4F54AE553B54F0AA0
:10213F00E554B55005C20802224BE553540744F04D
:10214F00F58385548263A20190637563A2017F08B2
:10215F00121D28906375E0F54BA3E0F54CE54C4557
:10216F004B70099080027410F07F0022906682E01D
:10217F00FFF46030906377E06F6003022212906685
:10218F0083E0FF906378E06F7079906684E0FF9052
:10219F006379E06F706D906685E0FF90637AE06F12
:1021AF006031805F906377E0906682F0906378E0B3
:1021BF00906683F0906379E0906684F090637AE0A4
:1021CF00906685F090637BE0FFA3E0906349CFF0CA
:1021DF00A3EFF0906375E0702AA3E024F8F54AE5C9
:1021EF0053540744F0F58385548274082582F58291
:1021FF00E43583F58363A20190637563A201AF4A4F
:10220F00121D28AE4BE4FCFDE554254CF554E55367
:10221F003EF553ED3552F552EC3551F551AF50AE09
:10222F004FAD4EAC4DAB54AA53A952A851D3121A6D
:10223F000040099080027410F07F002290802CE5FE
:10224F0051F0A3E552F0A3E553F0A3E554F09080CD
:06225F00027440F0AF4ADA
:012265002256
:1023E7009081E3E0F54A054A054A054A054A054A48
:1023F700054A054A054A054A054A90801CE0F54DFD
:10240700A3E0F54EA3E0F54FA3E0F5509081E4E09B
:10241700F54A054A054A054A054A054A054A054A4D
:10242700054A054A054A908020E0F551A3E0F55298
:10243700A3E0F553A3E0F554E4F54AE553B54F0A95
:10244700E554B55005C20902252EE553540744E863
:10245700F58385548263A20190600463A2017F0E15
:10246700121D3E906004E0F54BA3E0F54C90600C24
:10247700E0FFF4604390667BE0FEEF6E706AA3E0D6
:10248700FF90600DE06F706090667DE0FF90600EDA
:10249700E06F705490667EE0FF90600FE06F7048C9
:1024A70090667FE0FF906010E06F703C906680E080
:1024B700FF906011E06F7030906004E0702AA3E035
:1024C70024F2F54AE553540744E8F58385548274AA
:1024D7000E2582F582E43583F58363A201906004BB
:1024E70063A201AF4A121D3EAE4BE4FCFDE5542545
:1024F7004CF554E5533EF553ED3552F552EC355155
:10250700F551AF50AE4FAD4EAC4DAB54AA53A95297
:10251700A851D3121A005006E54C454B700990801C
:10252700017410F07F0022908020E551F0A3E5525E
:10253700F0A3E553F0A3E554F09080017440F0AFA9
:012547004A49
:012548002270
:0429C4008E4F8F5053
:1029C800908000E030E5079065787401F022906A05
:1029D80002E0FCA3E0FDA3E0FEA3E0F5568E558DD2
:1029E800548C53E556FFE5555407FEE42FF552EE97
:1029F80034C0F551855282F5837423F00552E552AF
:102A0800700205515351C7F582855183740AF00548
:102A180052E552700205515351C790633E63A201BB
:102A280085518385528263A2017F06121CE27406D7
:102A38002552F552E43551F551854F83855082630F
:102A4800A20185518385528263A201121CC6E4FC4F
:102A5800FDFE906A02E0F8A3E0F9A3E0FAA3E02FF4
:102A6800FFEE3AFEED39FDEC38FCEF2408FFE43EBA
:102A7800FEE43DFDE43CFC906A02121A11906A02E1
:102A8800E0908040F0906A03E0908041F0906A0402
:102A9800E0908042F0906A05E0908043F0908000DA
:032AA8007420F0A7
:012AAB002208
:0A27B9008E4F8F508C518D528B53C0
:1027C300908000E030E5079065787401F022906A0C
:1027D30002E0FCA3E0FDA3E0FEA3E0F5598E588DD3
:1027E300578C56E559FFE5585407FEE42FF555EE8F
:1027F30034C0F554855582F5837423F00555E555AA
:10280300700205545354C7F582855483740AF00546
:1028130055E555700205545354C790633E63A201B6
:1028230085548385558263A2017F06121CE27406D8
:102833002555F555E43554F554854F83855082630A
:10284300A20185548385558263A201121CC68F5A47
:10285300EF2555F555E43554F554E5536017855187
:102863008385528263A20185548385558263A201C5
:10287300AF53121CE2E55A24082553F553FFE4FC39
:10288300FDFEE5592FF559EE3558F558ED3557F559
:1028930057EC3556F556908040E556F0A3E557F0D2
:1028A300A3E558F0A3E559F09080007420F0AF59E8
:0C28B300AE58AD57AC56906A02121A11D4
:0128BF0022F6
:062B8D008E4B8F4C8D4DB4
:102B9300908000E030E5079065787401F022906A38
:102BA30002E0FCA3E0FDA3E0FEA3E0F5538E528D0B
:102BB300518C50E553FFE5525407FEE42FF54FEED9
:102BC30034C0F54E854F82F5837423F0054FE54FEE
:102BD3007002054E534EC7F582854E83EBF0054FC9
:102BE300E54F7002054E534EC790633E63A20185C5
:102BF3004E83854F8263A2017F06121CE274062571
:102C03004FF54FE4354EF54E854B83854C8263A2D9
:102C130001854E83854F8263A201AF4D121CE2747E
:102C230008254DF54DFFE4FCFDFEE5532FF553EE6E
:102C33003552F552ED3551F551EC3550F550908044
:102C430040E550F0A3E551F0A3E552F0A3E553F0BE
:102C53009080007420F0AF53AE52AD51AC50906AE7
:042C630002121A112E
:012C6700224A
:02335B008F637E
:10335D00908000E030E5079065787401F022906A66
:10336D0002E0FCA3E0FDA3E0FEA3E0F5678E668D11
:10337D00658C64E567FFE5665407FEE42FFFEE34C8
:10338D00C09062B463A201F5838F8263A201AF6323
:10339D00121CE2E4FCFDFEE5672563F567EE35667C
:1033AD00F566ED3565F565EC3564F564908040E5C1
:1033BD0064F0A3E565F0A3E566F0A3E567F0908002
:1033CD00007420F0AF67AE66AD65AC64906A021212
:0233DD001A11C3
:0133DF0022CB
:062AAC008E4D8F4EAB05BC
:102AB200908000E030E5079065787401F022906A1A
:102AC20002E0FCA3E0FDA3E0FEA3E0F5548E538DEB
:102AD200528C51E554FFE5535407FEE42FF550EEB6
:102AE20034C0F54F855082F5837423F00550E550CC
:102AF2007002054F534FC7F582854F83EBF00550A7
:102B0200E5507002054F90633E63A201854F8385B5
:102B1200508263A2017F06121CE274062550F55012
:102B2200E4354FF54F534FC7E54D855082854F83AE
:102B3200F00550E5507002054F534FC7F582854F9F
:102B420083E54EF00550E5507002054F534FC7E53F
:102B520054240AF554E43553F553E43552F552E45E
:102B62003551F551908040E551F0A3E552F0A3E5CF
:102B720053F0A3E554F09080007420F0AF54AE53AC
:0A2B8200AD52AC51906A02121A1114
:012B8C002226
:103B4F00A2AF921AC2AF438E2075D2028F828E839C
:0C3B5F00E0FFE4F5D2538EDFA21A92AF13
:013B6B002237
:103A7A00E5D220E0FBA2AF921AC2AF43D2028F82F4
:103A8A008E83EDF075D25063D250A21A92AFE5D26E
:033A9A0020E0FB2E
:013A9D002206
:1034E800E4FDED2401FFE433FE123B4F74362DF565
:1034F80082E43463F583EFF00DBD3FE6E4FDED248F
:103508007FFFE433FE123B4F742D2DF582E43461C6
:10351800F583EFF0742D2DF582E43461F583E070C6
:103528001B742D2DF582E43461F5837420F0742E1C
:103538002DF582E43461F583E4F080040DBD80BE8E
:10354800E49061ACF0FDEDFF7E00123B4F74AD2DB1
:0D355800F582E43461F583EFF00DBDFEE96E
:013565002243
:0239ED008B4FFE
:1039EF00A2AF921AC2AF85A25053A2FE8E838F82CE
:1039FF0005A28C838D827409121D6CE54F53A2FEB4
:103A0F0043A220121D6E53A2DF8550A2A21A92AFBD
:013A1F00FFA7
:013A20002283
:103B6C00A2AF921AC2AF8C838D82EF121D6C43A24E
:0C3B7C0020121D6E53A2DFA21A92AFFFB0
:013B8800221A
:023A9E008F4A4D
:103AA000A2AF921AC2AFE4F5838D827406121D6C28
:103AB000E54A43A220121D6E53A2DFA21A92AF7FE5
:013AC0000104
:013AC10022E2
:023AC2008F4A29
:103AC400A2AF921AC2AFE4F5838D82740A121D6C00
:103AD400E54A43A220121D6E53A2DFA21A92AF7FC1
:013AE40001E0
:013AE50022BE
:101B9500A907E7FFA805EF93C3966008403B74FCCF
:101BA5002FFF80F00F08EF93C3966008402B74FB5E
:101BB5002FFF80E00F08EF93C3966008401B74FA6F
:101BC5002FFF80D00F08EF93D3966008400B74F970
:101BD5002FFF80C01F1F1F1F1FEF54FEF80303F7C1
:101BE500E893FC08E893FD08E893FE08E893FF22D4
:101BF50009E993C39D6008402974FB29F980F1091F
:101C0500E993C39E6008401A74FA29F980E209E94C
:101C150093D39F6008400B74F929F980D3191919DA
:101C25001919E9C313C313FF22740093F8ECC39881
:101C35004024701F740193F8EDC398401970147413
:0E1C45000293F8EEC398400E7009740393F8F2
:101C5300EFC39840037F00227F0122EDF8E6F008EE
:101C6300A3DFFA22EDF8E0F608A3DFFA22E0A3638C
:101C7300A201F0A363A201DFF475A2002263A20113
:101C8300F0A363A20122E0A363A201F0A363A20174
:101C9300E0A363A201F0A363A201E463A201F0A3A2
:101CA30063A201DFE175A20022E0A363A2016DFE3E
:101CB300936CFDEE058393FC158363A201DFEA7544
:101CC300A200227F00E493A363A201F00F600CA3A0
:101CD300E583C2E3F58363A20180EA75A20022E0F3
:101CE300A363A201F0A3E583C2E3F58363A201DF4B
:101CF300EE75A20022E0A363A201F0A3E583C2E490
:101D0300D2E3F58363A201DFEC75A20022E0A363B3
:101D1300A201F0A3E58344F8C2E5F58363A201DFE2
:101D2300EC75A20022E583C2E3F583E0A363A2017D
:101D3300F0A363A201DFEE75A20022E583C2E4D221
:0A1D4300E3F583E0A363A201F0A31F
:101D4D0063A201DFEC75A20022E58344F8F583E080
:101D5D00A363A201F0A363A201DFEE75A20022F935
:101D6D0022C002C004C00612FFF0D006D004D0027B
:011D7D002243
:103857002043616E457247495400200A0045727241
:103867004C656E43616E21000A002043616E45720C
:1038770072434821000A205265714572722100C2C5
:1038870000C201C202C203C204C205C206C20700C7
:103897000000000000000000000000000000000021
:1038A7000000000000000000000000000000000011
:0138B7000010
:10254900E59B541F6020200B1A7E387F571229C43F
:10255900E59B541FFF7E007D03122AAC7E387F6104
:102569001229C4E4F59BE5BA30E010E4F5B375B17E
:1025790080F5B2D216F53A9067D7F0E5CFF470033B
:10258900022690754C01E4F54BE5CFF4554C7003E8
:1025990002267EE54BC454F0F5B1E5B2547F6420C0
:1025A900600302264FE5B3540FF52C85BC28E5BD21
:1025B900541FFF131313541FFFE5BD54E044184F74
:1025C900F529E5BDC43354E0FFE5BE131313541FC9
:1025D9004FF52AE5BEC43354E0FFE5BF1313135486
:1025E9001F4FF52B85A32D85A32E85A32F85A330FA
:1025F90085A33185A33285A33385A334E4F5B220BD
:10260900110CE528547EB5280575B350800375B3C0
:10261900D0301108E52830E7037F0022E52CD39458
:1026290008401D200B177E387F641229C4AF2C7E09
:10263900007D03122AAC7E387F6F1229C47F0022E5
:10264900E52C2405FF22E5B2549F6023200B207E50
:10265900387F711229C4AFB27E007D03122AACAF54
:10266900B37E007D03122AAC7E387F6F1229C4E441
:10267900F5B275B3D0E54C25E0F54C054BE54BC3F8
:09268900940850030225927F0021
:012692002225
:1037F5009066A1E0C39464505675B180E4F5B3F5C5
:10380500B28528BCE52AC4135407FFE52954E04FC7
:10381500F5BDE52A33333354F8FFE52BC4135407BC
:103825004FF5BEE52B33333354F8F5BF852DA3850E
:103835002EA3852FA38530A38531A38532A3853398
:10384500A38534A3E52C540F2450F5B3753A0AC269
:02385500162239
:102E020075B190E5B220E613200B107E387F7C125C
:102E120029C4AFB27E007D03122AACE4F5B3F5B249
:102E22007424250FF582E43467F583E0701B906902
:102E3200FDE0FFC31324E4F582E43469F583E07016
:102E420005430F808003430F40E50F30E615E4F59C
:102E52000F9069FDE02402F0E090388693700490B0
:102E620069FDF0E50F30E7219069FDE0FF903886BB
:102E720093F5BCE4F5BDEFA393FF33333354F8F578
:102E8200BE75BF78430F4080367424250FF582E467
:102E92003467F583E0F5BCE4F5BD7425250FF582B2
:102EA200E43467F583E0FF33333354F8F5BE75BF7E
:102EB20078050F050FE50FC394324003E4F50F7553
:032EC200B35022E8
:09002600EF6003C29622D296227B
:1034640043AB01C2E8C2EAE4FFEFC454F0F5B1C3D0
:10347400EF64809488500575B3D08003E4F5B3E419
:10348400F5B2F5BCF5BDF5BEF5BFF5C4F5C5F5C699
:10349400F5C7F5A3F5A3F5A3F5A3F5A3F5A3F5A344
:1034A400F5A30FBF0EC39066A1E0FE25E0F5B47549
:1034B400B50C75B66C75A11275AB0275C13E75C3BA
:1034C400FF75C203E49069FDF0750F80FF7F1990CA
:1034D40069E4E4F0A3DFFCE4FF7F32906724E4F0C6
:0334E400A3DFFC67
:0134E70022C2
:101D7E003E2A2C312CCFE0F0E0ECE5F2F0FB20E433
:101D8E00E8F1EFE5F2F7E5F0F1EAE8E3EE20F9E845
:101D9E00F2E00A003E4C2C4930312C256C752CD1CA
:101DAE00EAEEF0EEF1F2FC20EEE1ECE5EDE020EDF6
:101DBE00E020F8E8EDE52052533438352C3132303E
:101DCE00302C323430302C343830302C39363030F0
:101DDE002C31393230302C33383430302C353736D4
:101DEE0030302C3131353230300A003E4C2C4930F7
:101DFE00322C25732C43EAEEF0EEF1F2FC20EDE0EE
:101E0E0020F8E8EDE52043414E2C30202D203530D2
:101E1E0030EAE1283530EC292C31202D203530EAFE
:101E2E00E128353030EC292C32202D20D8E8EDE099
:101E3E0020EEF2EBFEF7E5EDE00A0030202D203526
:101E4E003030EAE1283530EC290031202D203530B4
:101E5E00EAE128353030EC290032202D20D8E8ED8B
:101E6E00E020EEF2EBFEF7E5EDE0003E532C4930BC
:101E7E00332C2562752CCFE5F0E8EEE420E8EDE496
:101E8E00E8EAE0F6E8E820282A3130ECF129283C8F
:101E9E00323530290A003E532C4930342C256275D8
:101EAE002CCFE5F0E8EEE420ECEEF0E3E0EDE8FF19
:101EBE0020282A3130ECF129283C323530290A000D
:101ECE003C21003C4930313D003C4930323D003C24
:101EDE004930333D003C4930343D000A41734F5583
:101EEE00543A000A4970496E3A000A546F43414E03
:101EFE003A00205265496E69742043414E0A002013
:101F0E0043414E283029203E20544F210A00D1F261
:101F1E00E0F0F220F1EAE0EDE8F0EEE2E0EDE8FFCD
:0D1F2E000A000A4173796E634B65793A0031
:103B0A00E4F5D975DE31F5E9F5F9F5ECF5FCF5EEF4
:103B1A00F5FEF544F5469067D6F075D84075B7407E
:033B2A00D2AE22F6
:0300330002226640
:0F226600C0E0C083C082C0D075D000C006C007E2
:1022750030DC1D85FE6885EE6974A12569F56974F4
:10228500133568F5688569EC8568FCC2DC75DC4941
:1022950020DA030223DAA297929385FC6885EC691C
:1022A50074422569F56974273568F5688569EC8593
:1022B50068FCE54414603414603E24FE7003022378
:1022C500D3240460030223D83097089067D6E0042E
:1022D500F080059067D6E4F09067D6E0D3940A5075
:1022E500030223D8E4F005440223D83097030223E0
:1022F500D8D29505440223D8E526C313F526309791
:10230500042480F5260546E546540760030223D8D4
:10231500E546131313541FFF24D7F582E43468F5FB
:1023250083E526F0BF03067544000223D8EF640653
:1023350070469068DBE0FF9068D8E0B5071D9068AF
:10234500DCE0FE9068D9E0B506119068DDE0FE900E
:1023550068DAE0B506057544008078754400906834
:10236500D8EFF09068DCE09068D9F09068DDE090F7
:1023750068DAF0754618805BE546131313541F643D
:102385000970469068DEE0FF9068D8E0B5071D90BB
:1023950068DFE0FE9068D9E0B506119068E0E0FEE0
:1023A5009068DAE0B506057544038027754400900A
:1023B50068D8EFF09068DFE09068D9F09068E0E0C9
:1023C5009068DAF0754618800A75440480057544EE
:0523D50001C295C2DA0F
:0D23DA00D007D006D0D0D082D083D0E03222
:102F75007BFF7A1D797E12136D9069E2E0FEA3E076
:102F8500FFC3E49FFFE49EFEAB07FA3395E0F9F833
:102F95007F007E8C7D0A7C001219608F558E548DC2
:102FA500538C527BFF7A1D79A212136D9066A1E0B6
:102FB50070127552FF75531E7554497BFF7A1D7942
:102FC500F912136D9066A1E0B40A127552FF75539C
:102FD5001E7554587BFF7A1D79F912136D9066A101
:102FE500E0B464127552FF75531E7554677BFF7A02
:102FF5001D79F912136D7BFF7A1E7979853B521283
:0F300500136D7BFF7A1E79A485385212136D224A
:103014007E1E7FCE1232D6EF4E70037F01227E1EBB
:103024007FD11232D6EF4E60231238B8A804A90516
:10303400AA06AB077F007E8C7D0A7C001219601201
:1030440019F29069E2EEF0A3EFF0800A9069E2745D
:10305400FFF0A374B8F0E49066A1F07E1E7FD7124F
:1030640032D6EF4E6015123B89BF31069066A174CB
:103074000AF0BF32069066A17464F07E1E7FDD12F2
:1030840032D6EF4E60071238B88F3B8003753B642D
:103094007E1E7FE31232D6EF4E60071238B88F38A7
:0730A400800375385A7F001C
:0130AB002202
:03002300022C6844
:0D2C6800C0E0C0F0C083C082C0D075D0189D
:102C7500309841C298AF9920120BEF64027035D29B
:102C850012D291802F301707C217531F0F8016BF1E
:102C95000904D217801EBF030C853E42753E00C253
:102CA50012C291800F74D8253EF582E43467F5830E
:102CB500EFF0053E30997130136CE53FB4FF0C75AC
:102CC5009902053F754500D290805BE53FB53D0B08
:102CD500C212C291759903053F804BE53FD3953DDF
:102CE500400DC213D219E4FF120026C2908037E5C9
:102CF500456009F599053F754500802A74E2253F31
:102D0500F582E43468F583E0F5456402600BE5453A
:102D150064036005E545B40905759909800885458D
:082D250099053F754500C299B4
:0B2D2D00D0D0D082D083D0F0D0E032B4
:1036C400E4FF120026C213C219C212C217E4F53F66
:1036D400F53DF53E9069E274FFF0A374F4F0E490D4
:1036E40066A3F0F50F9066A1F0753B6475385A1225
:1036F4003014C2ADE4F5C9D2CDD2CCC2C9C2CAF528
:10370400CDF5CC9069E2E0F5CBA3E0F5CA85CBCD4D
:1037140085CACCD29ED29CD2CAC2ACC298C2997578
:08372400B81075B710D2AC22F9
:0100210022BC
:02372C008F4BC1
:10372E00E4FFFEEEC3954B502874792EF582E434F7
:10373E0063F583E0FD74E22EF582E43468F583EDE3
:10374E00F074E22EF582E43468F583E02FFF0E80EC
:10375E00D2EFF4FF74E2254BF582E43468F583EF83
:10376E00F07F01120026E54B04F53D753FFFD213A5
:10377E00D299200B0C7E1E7FE97C687DE2FB12271E
:03378E00B9C219A4
:013791002215
:103B2D00300008C2009066A2E004F030130E9066DB
:103B3D00A2E0D39414400AC213D21922E49066A2D3
:023B4D00F02264
:03001E00E4FF22DA
:103A5400C28DC2AF438901C28C9066A1E0FF70079A
:103A6400F58A758CEE800AEFB40A06E4F58A758C43
:063A740070D28CD2AF22DB
:103A2100C28DC2AF438901C28C9066A1E0FF7014C0
:103A3100301809F58A758CDCC2188012758A667592
:103A41008CFC800AEFB40A06E4F58A758CDCD28C12
:033A5100D2AF22CF
:103AE6009066A1E0C394645006123464123A5412EC
:103AF6000021D216E4F53A9067D7F0F525F548C2CD
:043B060018F541224B
:02269300AB0793
:10269500EB24FCF54A200B0B7E1E7FF17C637D75D8
:1026A5001227B9906378E0641F600302279F906347
:1026B50075E0B40106AF4A12372C2290637BE064C3
:1026C5000870459067567442F0A37418F0906379CA
:1026D500E0FFC4540F906758F0EFC454F0FF9063C7
:1026E5007AE0FEC4540F2F906759F0A37408F09058
:1026F500637C63A20190675B63A201FF121C707586
:10270500250DE4F537C2142290637BE0FFB40A1D62
:102715009067567401F0A37418F0A37480F0A37445
:102725000AF0E4A3F0752505F537C21422EFB40BC2
:102735001D9067567401F0A37418F0A37480F0A37C
:102745007409F0E4A3F0752505F537C21422EFB43A
:102755000D1D9067567401F0A37418F0A37480F0F2
:10276500A3740BF0E4A3F0752505F537C21422EF29
:102775006407703F90675604F0A37418F0A3748043
:10278500F0A3740CF0A37401F090637CE090675B98
:10279500F0752506E4F537C2142290637963A2012A
:1027A50090675663A201AF4A121C70854A25E4F56D
:0327B50037C21414
:0127B80022FE
:03002F008F4A22D3
:10166700208D030216EFC28D2016030217A8E52569
:10167700604C90675AE02405F54AE4F525E54AD31E
:10168700940D4008D214123A540217A8906756E5F1
:101697004A540FFF7D28121C67E52830E702D2184D
:1016A700200B107E1E7FF87C677D56E54A540FFBA2
:1016B7001227B9123A541237F5D2140217A8E53C8B
:1016C700601790668D540FFF7D28121C67123A54DD
:1016D7001237F5E4F53C0217A89066A1E0C39464BD
:1016E7005003122E02123A541225498F4AEF700303
:1016F7000217A8123A21E4F541E547C3946E400367
:101707000217A82003030217A8E5286442706FE5B3
:101717002C7032E52AC454F0FFE52BC4540F2FF583
:1017270028E52BC454F0F529752A0874A42547F534
:1017370082E43466F58374032547F5477D287F03E4
:10174700121C5E805C74A42547F582E43466F58339
:10175700E54A2547F5477D28AF4A121C5E300D4103
:10176700C3E547954AFFE49400FE74A42FF58274FD
:10177700663EAF82FEE4FBAD4A122B8D8023E5283F
:10178700B44206E52B6402601874A42547F582E489
:101797003466F583E54A2547F5477D28AF4A121C8D
:1017A7005E300E1030000B9066A1E0C394645002C7
:1017B7000541C20E200203021920E53A6031D39495
:1017C700014004153A80289067D7E004F0E0D394ED
:1017D70003400D200B077E1F7F001229C4123AE633
:1017E700200B077E1F7F0D1229C4E4F53AD216E5B8
:1017F70043C394FD5002054320AE5520B33DE54356
:10180700D394FA4009E54394FE5003E4F543E543D6
:10181700640F60030218DC200B077E1F7F1C122950
:10182700C490637974FFF0A3F0A37409F07F0312E7
:10183700372C123B0AE4F5430218DCE543C3940A4C
:101847004008E543F460030218DC7543FD0218DC29
:10185700E54464037064200B0D7E1F7F307C687D38
:10186700D87B091227B9300D159068D87443F0E476
:10187700A3F0A3F07E687FD8FB7D06122B8D20B3E3
:10188700239068DBE0906379F09068DCE090637AFE
:10189700F0A37418F09068DDE090637CF07F041289
:1018A700372C801190637974FFF0A3F0A3740DF0C7
:1018B7007F0312372CC2AE7543FFE543B4FA169087
:1018C700637974FFF0A3F0A3740DF07F0312372C34
:1018D700C2AE7543FFE53C703E0539E539B53818AA
:1018E70090668D7401F0A37408F0A37480F0A3745C
:1018F70008F0E4A3F0753C05E539B53B1AE4F53982
:1019070090668D04F0A37408F0A37480F0A37407A5
:0C191700F0E4A3F0753C05C202123B2D69
:0119230022A1
:10365A00E5426033E4F54290647504F0A37403F024
:10366A0090667AE0906477F0A3741FF09067D8E0D0
:10367A00906479F09067D9E090647AF09067DAE024
:10368A0090647BF07F0122E547602CE4906475F03A
:10369A00A3E547F090667AE0906477F0A3741FF090
:1036AA009066A463A20190647963A201AF47121CD9
:0A36BA0070E4F5477F01227F002233
:103BA300301405C2147F0222301905C2197F032283
:033BB3007F00226E
:0100220022BB
:063BCD00E4F547F5252296
:0100320022AB
:10314800020863E493A3F8E493A34003F68001F232
:1031580008DFF48029E493A3F85407240CC8C33388
:10316800C4540F4420C8834004F456800146F6DF57
:10317800E4800B0102040810204080903BC6E47EE6
:10318800019360BCA3FF543F30E509541FFEE4934C
:10319800A360010ECF54C025E060A840B8E493A313
:1031A800FAE493A3F8E493A3C8C582C8CAC583CA3E
:1031B800F0A3C8C582C8CAC583CADFE9DEE780BEF6
:013BCC0000F8
:1019240075F008758200EF2FFFEE33FECD33CDCC7A
:1019340033CCC58233C5829BED9AEC99E5829840FD
:101944000CF582EE9BFEED9AFDEC99FC0FD5F0D6DA
:10195400E4CEFBE4CDFAE4CCF9A88222B800C1B904
:101964000059BA002DEC8BF084CFCECDFCE5F0CB42
:10197400F97818EF2FFFEE33FEED33FDEC33FCEB7B
:1019840033FB10D703994004EB99FB0FD8E5E4F936
:10199400FA227818EF2FFFEE33FEED33FDEC33FC23
:1019A400C933C910D7059BE99A4007EC9BFCE99A17
:1019B400F90FD8E0E4C9FAE4CCFB2275F010EF2F5C
:1019C400FFEE33FEED33FDCC33CCC833C810D7075C
:1019D4009BEC9AE899400AED9BFDEC9AFCE899F897
:0E19E4000FD5F0DAE4CDFBE4CCFAE4C8F9222A
:0E19F200C3E49FFFE49EFEE49DFDE49CFC2206
:101A0000EB9FF5F0EA9E42F0E99D42F0E89C45F03C
:011A100022B3
:0C1A1100ECF0A3EDF0A3EEF0A3EFF02248
:101A1D00A8828583F0D083D082121A34121A341220
:101A2D001A34121A34E473E493A3C583C5F0C58345
:101A3D00C8C582C8F0A3C583C5F0C583C8C582C813
:011A4D002276
:10130B00E55E2452F8E6055E22784F3021027852D2
:10131B00E475F001121AF5021A4E201AEB7F2ED249
:10132B001A8018EF540F2490D43440D4FF301E0B86
:10133B00EF24BFB41A0050032461FFE55F60021570
:10134B005F0562E5627002056130210D784FE4752F
:10135B00F001121AF5EF021A9402396E7403D221BE
:10136B008003E4C221F55E8B4F8A508951E4F55F0F
:10137B00F561F562E55F60077F2012134680F57516
:10138B0060FFC21BC21AC21CC21DC21FC220C222D6
:10139B00121314FF700D3021057F00121357AF622B
:1013AB00AE6122B4255FC2D5C21E121314FF24D026
:1013BB00B40A00501A75F00A785F30D50508B6FFED
:1013CB000106C6A426F620D5047002D21D80D924AE
:1013DB00CFB41A00EF5004C2E5D21E021557D21B30
:1013EB0080C6D21A80C0D21C80BCD2D580BAD21F84
:1013FB0080B47F20121346201C077401B55F004098
:10140B00F112130BFF12134602137FD222D220804C
:10141B009512130BFB12130BFA12130BF94A4B70A9
:10142B000679287A167BFF201C2EE55F602A7E004A
:10143B008E82758300121A6760060EEE656070F07F
:10144B00C2D5EBC0E0EAC0E0E9C0E0EE12159ED0D9
:10145B00E0F9D0E0FAD0E0FB121A4EFF60AAEBC025
:10146B00E0EAC0E0E9C0E0121346D0E02401F9D075
:10147B00E03400FAD0E0FBE5600460DCD560D98095
:10148B00877BFF7A15799AD21C809C791080027920
:10149B0008C220C2228008D2D5790A8004790AC2F8
:1014AB00D5E560047002F560E4FAFDFEFF12130B44
:1014BB00FC7B08201B1312130BFD7B10301A0A1236
:1014CB00130BFE12130BFF7B20EC3382D592D550FE
:1014DB0013C3E4301A069FFFE49EFEE4201B039D1A
:1014EB00FDE49CFCE4CBF8C21BEC700CCFCECDCC56
:1014FB00E824F8F870F38017C3EF33FFEE33FEEDFB
:10150B0033FDEC33FCEB33FB994002FB0FD8E9EBDB
:10151B00301B05F8D0E0C448B21BC0E00AEC4D4EBE
:10152B004F78207B0070C2EAB5600040BCC0E0126F
:10153B0015A0D0F0D0E0201B04C4C0E0C4B21BC087
:10154B00F012132FD0F0D5F0EB02137F121B5414B3
:10155B001C5314965813ED4C13E942149A4F14A2D2
:0F156B004414A24914024314A855148C46148C3E
:10157A0045148C4716485013F12D13F52E14182BC9
:10158A0013F92314162016312A13B1480000141037
:10159A003F3F3F00790AA2D5201D14301F09B91018
:1015AA00020404B9080104A2D52020025001042033
:1015BA001C68921CB55F005034C0E07F20301D19B2
:1015CA007F30A21C7220721F500F1215F7C21CC264
:1015DA0020C21FC2227F30800F301F03E9C0E012F1
:1015EA001346301F03D0E0F9D0E0B55FCC301F17A7
:1015FA007F30B9100C1213467F58301E077F78804F
:10160A0003B90803121346301C057F2D0213467FC7
:10161A00202022F87F2B2020F322921C80CF286ED4
:10162A00756C6C2900D21B12130B301BF8C21B7885
:10163A005F30D50108F60213B12D504349581213F1
:10164A000B2403B405004001E490164393121337A8
:0D165A00743A121337D21D755F0402149606
:101F3B008B4A8A4B894CE4F556F555F554F553F518
:101F4B0051F552E54E454F454D6012EBC0E0EAC0EE
:101F5B00E0E9C0E0AB4DAA4EA94F121B05AB4A05F9
:101F6B004CE54CAA4B7002054B14F9121A4EF5575F
:101F7B00C394094007E557D3940D40E1E55764201E
:101F8B0060DBE557B42D054352038016E557B42BA0
:101F9B0005435201800C74FF254CF54C74FF354BF7
:101FAB00F54BE55060046410703FAB4AAA4BA94C4B
:101FBB00121A4E64306009E550702E75500A802954
:101FCB00900001121A67FF64786004EFB458134352
:101FDB0052017550107402254CF54CE4354BF54B02
:101FEB008007E5507003755008AB4A054CE54CAAC9
:101FFB004B7002054B14F9121A4EF557C3946140FE
:10200B000AE557D3947A50035357DF74D02557F50D
:10201B0057C3940A400CE5579411406D74F925573A
:10202B00F557E557D39550506043520185565B8564
:10203B00555A855459855358AF507E00E4FCFDAB7F
:10204B0056AA55A954A853121AA6C8ECC8C9EDC96B
:10205B00CAEECACBEFCBE4FCFDFEEB2557F556EEF3
:10206B003AF555ED39F554EC38F553AF56AE55AD51
:10207B0054FCAB5BAA5AA959A858D3121A005003A7
:10208B00021FF4435204021FF4E55220E003E480E4
:10209B002DE54E454F454D601EAB4AE54C24FFF9EF
:1020AB00E54B34FFFAEBC0E0EAC0E0E9C0E0AB4D32
:1020BB00AA4EA94F121B05E55230E20774FFFFFE33
:1020CB00FDFC22E552AF56AE55AD54AC5330E10397
:0420DB000219F222D2
:101A4E00BB010689828A83E0225002E722BBFE0296
:091A5E00E32289828A83E49322C9
:101A6700BB010CE58229F582E5833AF583E0225034
:101A770006E92582F8E622BBFE06E92582F8E2227E
:0D1A8700E58229F582E5833AF583E4932298
:101A9400BB010689828A83F0225002F722BBFE0131
:021AA400F3222B
:101AA600E88FF0A4CC8BF0A42CFCE98EF0A42CFCDF
:101AB6008AF0EDA42CFCEA8EF0A4CDA8F08BF0A45D
:101AC6002DCC3825F0FDE98FF0A42CCD35F0FCEBBC
:101AD6008EF0A4FEA9F0EB8FF0A4CFC5F02ECD3981
:0F1AE600FEE43CFCEAA42DCE35F0FDE43CFC22EE
:101AF500FAE6FB0808E6F925F0F618E6CA3AF622F2
:101B0500BB011A89828A83D0F0D0E0F8D0E0F9D001
:101B1500E0FAD0E0FBE8C0E0C0F0021B835016E914
:101B2500F8D083D082D0E0F9D0E0FAD0E0FBC082D3
:101B3500C083021B7ABBFE16E9F8D083D082D0E0C1
:0F1B4500F9D0E0FAD0E0FBC082C083021B8C22F3
:101B5400D083D082F8E4937012740193700DA3A320
:101B640093F8740193F5828883E473740293686034
:061B7400EFA3A3A380DF34
:091B7A00EBF608EAF608E9F62290
:091B8300EBF0A3EAF0A3E9F02263
:091B8C00EBF208EAF208E9F2228A
:00000001FF
